:020000001128C5
:08000800102800006400000054
:020010000528C1
:10002000052896019801FF309000FE309200FE30C6
:100030009100BB20640000002F20161920282428DE
:10004000051585118514272885150511851099201A
:100050001008970017080B3A031998011A2810087E
:100060009700861106158614CD20061A3A2801300D
:1000700090008428861A3F28043090008428061BAC
:100080004428073090008428861B49280A309000B5
:100090008428861506118614CD20061A52280230AF
:1000A00090008428861A5728053090008428061B63
:1000B0005C28083090008428861B6128003090005E
:1000C0008428861506158610CD20061A6A28033066
:1000D00090008428861A6F28063090008428061B1A
:1000E0007428093090008428861B79280B309000F2
:1000F000842816187C287F28170890008128FF3054
:100100009000161085118928161C8D2000001614E9
:1001100085158615061586140800980A2108A00082
:100120002208A1002308A2002408A3001008A400AC
:100130000800200897001708013A031DB928210874
:1001400097001708083A031DB928220897001708D6
:10015000083A031DB928230897001708013A031D20
:10016000B9282408970017080B3A031DB92816155B
:10017000BA2816110800860185018316F130860021
:10018000103085008113831208006400C830940089
:10019000D128640014309400D12864000230940007
:1001A000D128A8309500950BD328940BD1280800AE
:02400E00F73F7A
:00000001FF
